:06000000116A77EF3EF0EB
:107C0400F26AD06A1200C586C7A0FED7C950120016
:107C1400E8CFD9FF9EA8FED7D9CFADFF1200E8CF99
:107C2400D9FF3F0EC716C66AC56AD950C6121D5081
:107C3400C71293829380C68A1200E8CFD9FF040E3C
:107C4400E96EFA0E106E000100F000F000F000F092
:107C540000F000F000F000F000F0102F26EF3EF0EE
:107C640000F0E92EEED7D92EEAD7FA0CE8CFE9FFD7
:107C7400E9CFC9FFC6BE1200C7B0FED7C5CF1DF0FD
:107C84001F0E1D161DC01EF01F6A000EC7B4010E84
:107C94001E121F501E10F2E1C5BC120012001E502D
:107CA400D96E10D0D9061068000100F000F000F081
:107CB40000F000F000F000F000F000F0102F57EF9B
:107CC4003EF000F0010ED960EDD71DC010F00001A8
:107CD40000F000F000F000F000F000F000F000F020
:107CE40000F0102F6AEF3EF0010C02EC3EF0948E8F
:107CF400948C4D0EAF6E900EAB6E200EAC6E120EC9
:107D0400186E000E196E58EC3FF0120E186E000E2D
:107D1400196ED1EC3EF0FF0E0AEC3EF0C80E106E68
:107D2400000100F000F000F000F000F000F000F0BE
:107D340000F000F0102F93EF3EF0000E0AEC3EF03E
:107D4400C80E106E000100F000F000F000F000F02A
:107D540000F000F000F000F0102FA5EF3EF0E16A13
:107D6400120EE124E96EEA6A000EEA22EF50170AC5
:107D7400170F0AEC3EF0C80E106E000100F000F080
:107D840000F000F000F000F000F000F000F0102F20
:107D9400C0EF3EF0E12A050EE164E2D7B6D7C58014
:107DA400C5CF1AF01F0E1A161AC01BF01C6A000E5B
:107DB400C7B4010E1B121C501B10F2E1A40E38ECC8
:107DC4003EF0C5CF1AF01F0E1A161AC01BF01C6A1B
:107DD400000EC7B4010E1B121C501B10F2E1000E62
:107DE40038EC3EF0C5CF1AF01F0E1A161AC01BF05D
:107DF4001C6A000EC7B4010E1B121C501B10F2E1CA
:107E0400C5849E0E106E000100F000F000F000F03A
:107E140000F000F000F000F000F0102F06EF3FF04B
:107E2400C580C5CF1AF01F0E1A161AC01BF01C6AA3
:107E3400000EC7B4010E1B121C501B10F2E1A50E5C
:107E440038EC3EF0116A1DD0C5CF1AF01F0E1A1679
:107E54001AC01BF01C6A000EC7B4010E1B121C5082
:107E64001B10F2E111501824E96E000E1920EA6E7D
:107E740005EC3EF0EF6E060E116002D0C59AC5887F
:107E8400112A050E1164E0D7C58AC588C5CF1AF03A
:107E94001F0E1A161AC01BF01C6A000EC7B4010E7E
:107EA4001B121C501B10F2E1C5841200C00E1D6E83
:107EB400080E11EC3EF0270EC86E140E1FEC3EF0B7
:107EC400C580C5CF1AF01F0E1A161AC01BF01C6A03
:107ED400000EC7B4010E1B121C501B10F2E1A40EBD
:107EE40038EC3EF0C5CF1AF01F0E1A161AC01BF05C
:107EF4001C6A000EC7B4010E1B121C501B10F2E1C9
:107F0400400E38EC3EF0C5CF1AF01F0E1A161AC0F8
:107F14001BF01C6A000EC7B4010E1B121C501B1070
:107F2400F2E1000E38EC3EF0C5CF1AF01F0E1A161F
:107F34001AC01BF01C6A000EC7B4010E1B121C50A1
:107F44001B10F2E1C584E60E1D6E030E1E6E51EC8D
:107F54003EF0C580C5CF1AF01F0E1A161AC01BF0CA
:107F64001C6A000EC7B4010E1B121C501B10F2E158
:107F7400A50E38EC3EF0116A1DD0C5CF1AF01F0EC5
:107F84001A161AC01BF01C6A000EC7B4010E1B128D
:107F94001C501B10F2E111501824E96E000E192038
:107FA400EA6E05EC3EF0EF6E060E116002D0C59A43
:107FB400C588112A050E1164E0D7C58AC588C5CFC6
:107FC4001AF01F0E1A161AC01BF01C6A000EC7B452
:107FD400010E1B121C501B10F2E1C5841B0E106E07
:107FE400000100F000F000F000F000F000F000F0FC
:0C7FF40000F000F0102FF3EF3FF01B0C2A
:020000040030CA
:0E000000E43FC0E0FFF8BAFFFFFFFFFFFFFF85
:00000001FF
